Component: ARM Compiler 5.06 update 7 (build 960) Tool: armlink [4d3601]

==============================================================================

Section Cross References

    main.o(.ARM.__at_0x20000100) refers to rt_memclr_w.o(.text) for __aeabi_memclr4
    main.o(.ARM.__at_0x20000100) refers to main.o(.bss) for .bss
    main.o(.ARM.__at_0x20000100) refers to main.o(.data) for .data
    startup.o(.startup) refers to main.o(.bss) for FlashParameter
    startup.o(.startup) refers to main.o(.ARM.__at_0x20000100) for main
    __main.o(!!!main) refers to __rtentry.o(.ARM.Collect$$rtentry$$00000000) for __rt_entry
    __rtentry.o(.ARM.Collect$$rtentry$$00000000) refers (Special) to __rtentry2.o(.ARM.Collect$$rtentry$$0000000A) for __rt_entry_li
    __rtentry.o(.ARM.Collect$$rtentry$$00000000) refers (Special) to __rtentry2.o(.ARM.Collect$$rtentry$$0000000D) for __rt_entry_main
    __rtentry.o(.ARM.Collect$$rtentry$$00000000) refers (Special) to __rtentry2.o(.ARM.Collect$$rtentry$$0000000C) for __rt_entry_postli_1
    __rtentry.o(.ARM.Collect$$rtentry$$00000000) refers (Special) to __rtentry2.o(.ARM.Collect$$rtentry$$00000009) for __rt_entry_postsh_1
    __rtentry.o(.ARM.Collect$$rtentry$$00000000) refers (Special) to __rtentry2.o(.ARM.Collect$$rtentry$$00000002) for __rt_entry_presh_1
    __rtentry.o(.ARM.Collect$$rtentry$$00000000) refers (Special) to __rtentry4.o(.ARM.Collect$$rtentry$$00000004) for __rt_entry_sh
    __rtentry2.o(.ARM.Collect$$rtentry$$00000008) refers to boardinit2.o(.text) for _platform_post_stackheap_init
    __rtentry2.o(.ARM.Collect$$rtentry$$0000000A) refers to libinit.o(.ARM.Collect$$libinit$$00000000) for __rt_lib_init
    __rtentry2.o(.ARM.Collect$$rtentry$$0000000B) refers to boardinit3.o(.text) for _platform_post_lib_init
    __rtentry2.o(.ARM.Collect$$rtentry$$0000000D) refers to main.o(.ARM.__at_0x20000100) for main
    __rtentry2.o(.ARM.Collect$$rtentry$$0000000D) refers to exit.o(.text) for exit
    __rtentry2.o(.ARM.exidx) refers to __rtentry2.o(.ARM.Collect$$rtentry$$00000001) for .ARM.Collect$$rtentry$$00000001
    __rtentry2.o(.ARM.exidx) refers to __rtentry2.o(.ARM.Collect$$rtentry$$00000008) for .ARM.Collect$$rtentry$$00000008
    __rtentry2.o(.ARM.exidx) refers to __rtentry2.o(.ARM.Collect$$rtentry$$0000000A) for .ARM.Collect$$rtentry$$0000000A
    __rtentry2.o(.ARM.exidx) refers to __rtentry2.o(.ARM.Collect$$rtentry$$0000000B) for .ARM.Collect$$rtentry$$0000000B
    __rtentry2.o(.ARM.exidx) refers to __rtentry2.o(.ARM.Collect$$rtentry$$0000000D) for .ARM.Collect$$rtentry$$0000000D
    __rtentry4.o(.ARM.Collect$$rtentry$$00000004) refers to sys_stackheap_outer.o(.text) for __user_setup_stackheap
    __rtentry4.o(.ARM.exidx) refers to __rtentry4.o(.ARM.Collect$$rtentry$$00000004) for .ARM.Collect$$rtentry$$00000004
    sys_stackheap_outer.o(.text) refers to libspace.o(.text) for __user_perproc_libspace
    sys_stackheap_outer.o(.text) refers to sys_stackheap.o(.text) for __user_initial_stackheap
    exit.o(.text) refers to rtexit.o(.ARM.Collect$$rtexit$$00000000) for __rt_exit
    libinit.o(.ARM.Collect$$libinit$$00000000) refers (Special) to libinit2.o(.ARM.Collect$$libinit$$0000002E) for __rt_lib_init_alloca_1
    libinit.o(.ARM.Collect$$libinit$$00000000) refers (Special) to libinit2.o(.ARM.Collect$$libinit$$0000002C) for __rt_lib_init_argv_1
    libinit.o(.ARM.Collect$$libinit$$00000000) refers (Special) to libinit2.o(.ARM.Collect$$libinit$$0000001B) for __rt_lib_init_atexit_1
    libinit.o(.ARM.Collect$$libinit$$00000000) refers (Special) to libinit2.o(.ARM.Collect$$libinit$$00000021) for __rt_lib_init_clock_1
    libinit.o(.ARM.Collect$$libinit$$00000000) refers (Special) to libinit2.o(.ARM.Collect$$libinit$$00000032) for __rt_lib_init_cpp_1
    libinit.o(.ARM.Collect$$libinit$$00000000) refers (Special) to libinit2.o(.ARM.Collect$$libinit$$00000030) for __rt_lib_init_exceptions_1
    libinit.o(.ARM.Collect$$libinit$$00000000) refers (Special) to libinit2.o(.ARM.Collect$$libinit$$00000002) for __rt_lib_init_fp_1
    libinit.o(.ARM.Collect$$libinit$$00000000) refers (Special) to libinit2.o(.ARM.Collect$$libinit$$0000001F) for __rt_lib_init_fp_trap_1
    libinit.o(.ARM.Collect$$libinit$$00000000) refers (Special) to libinit2.o(.ARM.Collect$$libinit$$00000023) for __rt_lib_init_getenv_1
    libinit.o(.ARM.Collect$$libinit$$00000000) refers (Special) to libinit2.o(.ARM.Collect$$libinit$$0000000A) for __rt_lib_init_heap_1
    libinit.o(.ARM.Collect$$libinit$$00000000) refers (Special) to libinit2.o(.ARM.Collect$$libinit$$00000011) for __rt_lib_init_lc_collate_1
    libinit.o(.ARM.Collect$$libinit$$00000000) refers (Special) to libinit2.o(.ARM.Collect$$libinit$$00000013) for __rt_lib_init_lc_ctype_1
    libinit.o(.ARM.Collect$$libinit$$00000000) refers (Special) to libinit2.o(.ARM.Collect$$libinit$$00000015) for __rt_lib_init_lc_monetary_1
    libinit.o(.ARM.Collect$$libinit$$00000000) refers (Special) to libinit2.o(.ARM.Collect$$libinit$$00000017) for __rt_lib_init_lc_numeric_1
    libinit.o(.ARM.Collect$$libinit$$00000000) refers (Special) to libinit2.o(.ARM.Collect$$libinit$$00000019) for __rt_lib_init_lc_time_1
    libinit.o(.ARM.Collect$$libinit$$00000000) refers (Special) to libinit2.o(.ARM.Collect$$libinit$$00000004) for __rt_lib_init_preinit_1
    libinit.o(.ARM.Collect$$libinit$$00000000) refers (Special) to libinit2.o(.ARM.Collect$$libinit$$0000000E) for __rt_lib_init_rand_1
    libinit.o(.ARM.Collect$$libinit$$00000000) refers (Special) to libinit2.o(.ARM.Collect$$libinit$$00000033) for __rt_lib_init_return
    libinit.o(.ARM.Collect$$libinit$$00000000) refers (Special) to libinit2.o(.ARM.Collect$$libinit$$0000001D) for __rt_lib_init_signal_1
    libinit.o(.ARM.Collect$$libinit$$00000000) refers (Special) to libinit2.o(.ARM.Collect$$libinit$$00000025) for __rt_lib_init_stdio_1
    libinit.o(.ARM.Collect$$libinit$$00000000) refers (Special) to libinit2.o(.ARM.Collect$$libinit$$0000000C) for __rt_lib_init_user_alloc_1
    libspace.o(.text) refers to libspace.o(.bss) for __libspace_start
    sys_stackheap.o(.text) refers (Special) to indicate_semi.o(.text) for __semihosting_library_function
    sys_stackheap.o(.text) refers to use_no_semi.o(.text) for __I$use$semihosting
    rtexit.o(.ARM.Collect$$rtexit$$00000000) refers (Special) to rtexit2.o(.ARM.Collect$$rtexit$$00000004) for __rt_exit_exit
    rtexit.o(.ARM.Collect$$rtexit$$00000000) refers (Special) to rtexit2.o(.ARM.Collect$$rtexit$$00000003) for __rt_exit_ls
    rtexit.o(.ARM.Collect$$rtexit$$00000000) refers (Special) to rtexit2.o(.ARM.Collect$$rtexit$$00000002) for __rt_exit_prels_1
    rtexit.o(.ARM.exidx) refers (Special) to rtexit2.o(.ARM.Collect$$rtexit$$00000004) for __rt_exit_exit
    rtexit.o(.ARM.exidx) refers (Special) to rtexit2.o(.ARM.Collect$$rtexit$$00000003) for __rt_exit_ls
    rtexit.o(.ARM.exidx) refers (Special) to rtexit2.o(.ARM.Collect$$rtexit$$00000002) for __rt_exit_prels_1
    rtexit.o(.ARM.exidx) refers to rtexit.o(.ARM.Collect$$rtexit$$00000000) for .ARM.Collect$$rtexit$$00000000
    libinit2.o(.ARM.Collect$$libinit$$00000010) refers to libinit2.o(.ARM.Collect$$libinit$$0000000F) for .ARM.Collect$$libinit$$0000000F
    libinit2.o(.ARM.Collect$$libinit$$00000012) refers to libinit2.o(.ARM.Collect$$libinit$$0000000F) for .ARM.Collect$$libinit$$0000000F
    libinit2.o(.ARM.Collect$$libinit$$00000014) refers to libinit2.o(.ARM.Collect$$libinit$$0000000F) for .ARM.Collect$$libinit$$0000000F
    libinit2.o(.ARM.Collect$$libinit$$00000016) refers to libinit2.o(.ARM.Collect$$libinit$$0000000F) for .ARM.Collect$$libinit$$0000000F
    libinit2.o(.ARM.Collect$$libinit$$00000018) refers to libinit2.o(.ARM.Collect$$libinit$$0000000F) for .ARM.Collect$$libinit$$0000000F
    libinit2.o(.ARM.Collect$$libinit$$00000026) refers to argv_veneer.o(.emb_text) for __ARM_argv_veneer
    libinit2.o(.ARM.Collect$$libinit$$00000027) refers to argv_veneer.o(.emb_text) for __ARM_argv_veneer
    rtexit2.o(.ARM.Collect$$rtexit$$00000003) refers to libshutdown.o(.ARM.Collect$$libshutdown$$00000000) for __rt_lib_shutdown
    rtexit2.o(.ARM.Collect$$rtexit$$00000004) refers to sys_exit.o(.text) for _sys_exit
    rtexit2.o(.ARM.exidx) refers to rtexit2.o(.ARM.Collect$$rtexit$$00000001) for .ARM.Collect$$rtexit$$00000001
    rtexit2.o(.ARM.exidx) refers to rtexit2.o(.ARM.Collect$$rtexit$$00000003) for .ARM.Collect$$rtexit$$00000003
    rtexit2.o(.ARM.exidx) refers to rtexit2.o(.ARM.Collect$$rtexit$$00000004) for .ARM.Collect$$rtexit$$00000004
    argv_veneer.o(.emb_text) refers to no_argv.o(.text) for __ARM_get_argv
    sys_exit.o(.text) refers (Special) to use_no_semi.o(.text) for __I$use$semihosting
    sys_exit.o(.text) refers (Special) to indicate_semi.o(.text) for __semihosting_library_function
    _get_argv_nomalloc.o(.text) refers (Special) to hrguard.o(.text) for __heap_region$guard
    _get_argv_nomalloc.o(.text) refers to defsig_rtmem_outer.o(.text) for __rt_SIGRTMEM
    _get_argv_nomalloc.o(.text) refers to sys_command.o(.text) for _sys_command_string
    libshutdown.o(.ARM.Collect$$libshutdown$$00000000) refers (Special) to libshutdown2.o(.ARM.Collect$$libshutdown$$00000004) for __rt_lib_shutdown_cpp_1
    libshutdown.o(.ARM.Collect$$libshutdown$$00000000) refers (Special) to libshutdown2.o(.ARM.Collect$$libshutdown$$00000002) for __rt_lib_shutdown_fini_1
    libshutdown.o(.ARM.Collect$$libshutdown$$00000000) refers (Special) to libshutdown2.o(.ARM.Collect$$libshutdown$$00000009) for __rt_lib_shutdown_fp_trap_1
    libshutdown.o(.ARM.Collect$$libshutdown$$00000000) refers (Special) to libshutdown2.o(.ARM.Collect$$libshutdown$$00000011) for __rt_lib_shutdown_heap_1
    libshutdown.o(.ARM.Collect$$libshutdown$$00000000) refers (Special) to libshutdown2.o(.ARM.Collect$$libshutdown$$00000012) for __rt_lib_shutdown_return
    libshutdown.o(.ARM.Collect$$libshutdown$$00000000) refers (Special) to libshutdown2.o(.ARM.Collect$$libshutdown$$0000000C) for __rt_lib_shutdown_signal_1
    libshutdown.o(.ARM.Collect$$libshutdown$$00000000) refers (Special) to libshutdown2.o(.ARM.Collect$$libshutdown$$00000006) for __rt_lib_shutdown_stdio_1
    libshutdown.o(.ARM.Collect$$libshutdown$$00000000) refers (Special) to libshutdown2.o(.ARM.Collect$$libshutdown$$0000000E) for __rt_lib_shutdown_user_alloc_1
    sys_command.o(.text) refers (Special) to use_no_semi.o(.text) for __I$use$semihosting
    sys_command.o(.text) refers (Special) to indicate_semi.o(.text) for __semihosting_library_function
    defsig_rtmem_outer.o(.text) refers to defsig_rtmem_inner.o(.text) for __rt_SIGRTMEM_inner
    defsig_rtmem_outer.o(.text) refers to defsig_exit.o(.text) for __sig_exit
    defsig_rtmem_formal.o(.text) refers to rt_raise.o(.text) for __rt_raise
    rt_raise.o(.text) refers to __raise.o(.text) for __raise
    rt_raise.o(.text) refers to sys_exit.o(.text) for _sys_exit
    defsig_exit.o(.text) refers to sys_exit.o(.text) for _sys_exit
    defsig_rtmem_inner.o(.text) refers to defsig_general.o(.text) for __default_signal_display
    __raise.o(.text) refers to defsig.o(CL$$defsig) for __default_signal_handler
    defsig_general.o(.text) refers to sys_wrch.o(.text) for _ttywrch
    sys_wrch.o(.text) refers (Special) to use_no_semi.o(.text) for __I$use$semihosting
    sys_wrch.o(.text) refers (Special) to indicate_semi.o(.text) for __semihosting_library_function
    defsig.o(CL$$defsig) refers to defsig_rtmem_inner.o(.text) for __rt_SIGRTMEM_inner
    defsig_abrt_inner.o(.text) refers to defsig_general.o(.text) for __default_signal_display
    defsig_fpe_inner.o(.text) refers to defsig_general.o(.text) for __default_signal_display
    defsig_rtred_inner.o(.text) refers to defsig_general.o(.text) for __default_signal_display
    defsig_stak_inner.o(.text) refers to defsig_general.o(.text) for __default_signal_display
    defsig_pvfn_inner.o(.text) refers to defsig_general.o(.text) for __default_signal_display
    defsig_cppl_inner.o(.text) refers to defsig_general.o(.text) for __default_signal_display
    defsig_segv_inner.o(.text) refers to defsig_general.o(.text) for __default_signal_display
    defsig_other.o(.text) refers to defsig_general.o(.text) for __default_signal_display


==============================================================================

Removing Unused input sections from the image.

    Removing main.o(.constdata), (4 bytes).

1 unused section(s) (total 4 bytes) removed from the image.

==============================================================================

Image Symbol Table

    Local Symbols

    Symbol Name                              Value     Ov Type        Size  Object(Section)

    ../clib/angel/boardlib.s                 0x00000000   Number         0  boardinit1.o ABSOLUTE
    ../clib/angel/boardlib.s                 0x00000000   Number         0  boardinit2.o ABSOLUTE
    ../clib/angel/boardlib.s                 0x00000000   Number         0  boardinit3.o ABSOLUTE
    ../clib/angel/boardlib.s                 0x00000000   Number         0  boardshut.o ABSOLUTE
    ../clib/angel/handlers.s                 0x00000000   Number         0  __scatter_zi.o ABSOLUTE
    ../clib/angel/kernel.s                   0x00000000   Number         0  __rtentry.o ABSOLUTE
    ../clib/angel/kernel.s                   0x00000000   Number         0  rtexit.o ABSOLUTE
    ../clib/angel/kernel.s                   0x00000000   Number         0  __rtentry2.o ABSOLUTE
    ../clib/angel/kernel.s                   0x00000000   Number         0  __rtentry4.o ABSOLUTE
    ../clib/angel/kernel.s                   0x00000000   Number         0  rtexit2.o ABSOLUTE
    ../clib/angel/rt.s                       0x00000000   Number         0  rt_raise.o ABSOLUTE
    ../clib/angel/scatter.s                  0x00000000   Number         0  __scatter.o ABSOLUTE
    ../clib/angel/startup.s                  0x00000000   Number         0  __main.o ABSOLUTE
    ../clib/angel/sys.s                      0x00000000   Number         0  use_no_semi.o ABSOLUTE
    ../clib/angel/sys.s                      0x00000000   Number         0  sys_stackheap_outer.o ABSOLUTE
    ../clib/angel/sys.s                      0x00000000   Number         0  indicate_semi.o ABSOLUTE
    ../clib/angel/sys.s                      0x00000000   Number         0  libspace.o ABSOLUTE
    ../clib/angel/sys.s                      0x00000000   Number         0  sys_stackheap.o ABSOLUTE
    ../clib/angel/sysapp.c                   0x00000000   Number         0  sys_wrch.o ABSOLUTE
    ../clib/angel/sysapp.c                   0x00000000   Number         0  sys_command.o ABSOLUTE
    ../clib/angel/sysapp.c                   0x00000000   Number         0  sys_exit.o ABSOLUTE
    ../clib/armsys.c                         0x00000000   Number         0  no_argv.o ABSOLUTE
    ../clib/armsys.c                         0x00000000   Number         0  _get_argv_nomalloc.o ABSOLUTE
    ../clib/armsys.c                         0x00000000   Number         0  argv_veneer.o ABSOLUTE
    ../clib/armsys.c                         0x00000000   Number         0  argv_veneer.o ABSOLUTE
    ../clib/heapalloc.c                      0x00000000   Number         0  hrguard.o ABSOLUTE
    ../clib/libinit.s                        0x00000000   Number         0  libinit.o ABSOLUTE
    ../clib/libinit.s                        0x00000000   Number         0  libshutdown.o ABSOLUTE
    ../clib/libinit.s                        0x00000000   Number         0  libshutdown2.o ABSOLUTE
    ../clib/libinit.s                        0x00000000   Number         0  libinit2.o ABSOLUTE
    ../clib/memcpset.s                       0x00000000   Number         0  rt_memclr_w.o ABSOLUTE
    ../clib/signal.c                         0x00000000   Number         0  defsig_rtred_inner.o ABSOLUTE
    ../clib/signal.c                         0x00000000   Number         0  defsig_rtmem_inner.o ABSOLUTE
    ../clib/signal.c                         0x00000000   Number         0  __raise.o ABSOLUTE
    ../clib/signal.c                         0x00000000   Number         0  defsig_exit.o ABSOLUTE
    ../clib/signal.c                         0x00000000   Number         0  defsig_general.o ABSOLUTE
    ../clib/signal.c                         0x00000000   Number         0  defsig_rtmem_outer.o ABSOLUTE
    ../clib/signal.c                         0x00000000   Number         0  defsig_rtmem_formal.o ABSOLUTE
    ../clib/signal.c                         0x00000000   Number         0  defsig_abrt_inner.o ABSOLUTE
    ../clib/signal.c                         0x00000000   Number         0  defsig_other.o ABSOLUTE
    ../clib/signal.c                         0x00000000   Number         0  defsig_segv_inner.o ABSOLUTE
    ../clib/signal.c                         0x00000000   Number         0  defsig_cppl_inner.o ABSOLUTE
    ../clib/signal.c                         0x00000000   Number         0  defsig_pvfn_inner.o ABSOLUTE
    ../clib/signal.c                         0x00000000   Number         0  defsig_stak_inner.o ABSOLUTE
    ../clib/signal.c                         0x00000000   Number         0  defsig_fpe_inner.o ABSOLUTE
    ../clib/signal.s                         0x00000000   Number         0  defsig.o ABSOLUTE
    ../clib/stdlib.c                         0x00000000   Number         0  exit.o ABSOLUTE
    ../fplib/fpinit.s                        0x00000000   Number         0  fpinit.o ABSOLUTE
    dc.s                                     0x00000000   Number         0  dc.o ABSOLUTE
    main.c                                   0x00000000   Number         0  main.o ABSOLUTE
    startup.s                                0x00000000   Number         0  startup.o ABSOLUTE
    .startup                                 0x20000000   Section       60  startup.o(.startup)
    !!!main                                  0x2000003c   Section        8  __main.o(!!!main)
    !!!scatter                               0x20000044   Section       52  __scatter.o(!!!scatter)
    !!handler_zi                             0x20000078   Section       28  __scatter_zi.o(!!handler_zi)
    .ARM.Collect$$libinit$$00000000          0x20000094   Section        2  libinit.o(.ARM.Collect$$libinit$$00000000)
    .ARM.Collect$$libinit$$00000002          0x20000096   Section        0  libinit2.o(.ARM.Collect$$libinit$$00000002)
    .ARM.Collect$$libinit$$00000004          0x20000096   Section        0  libinit2.o(.ARM.Collect$$libinit$$00000004)
    .ARM.Collect$$libinit$$0000000A          0x20000096   Section        0  libinit2.o(.ARM.Collect$$libinit$$0000000A)
    .ARM.Collect$$libinit$$0000000C          0x20000096   Section        0  libinit2.o(.ARM.Collect$$libinit$$0000000C)
    .ARM.Collect$$libinit$$0000000E          0x20000096   Section        0  libinit2.o(.ARM.Collect$$libinit$$0000000E)
    .ARM.Collect$$libinit$$00000011          0x20000096   Section        0  libinit2.o(.ARM.Collect$$libinit$$00000011)
    .ARM.Collect$$libinit$$00000013          0x20000096   Section        0  libinit2.o(.ARM.Collect$$libinit$$00000013)
    .ARM.Collect$$libinit$$00000015          0x20000096   Section        0  libinit2.o(.ARM.Collect$$libinit$$00000015)
    .ARM.Collect$$libinit$$00000017          0x20000096   Section        0  libinit2.o(.ARM.Collect$$libinit$$00000017)
    .ARM.Collect$$libinit$$00000019          0x20000096   Section        0  libinit2.o(.ARM.Collect$$libinit$$00000019)
    .ARM.Collect$$libinit$$0000001B          0x20000096   Section        0  libinit2.o(.ARM.Collect$$libinit$$0000001B)
    .ARM.Collect$$libinit$$0000001D          0x20000096   Section        0  libinit2.o(.ARM.Collect$$libinit$$0000001D)
    .ARM.Collect$$libinit$$0000001F          0x20000096   Section        0  libinit2.o(.ARM.Collect$$libinit$$0000001F)
    .ARM.Collect$$libinit$$00000021          0x20000096   Section        0  libinit2.o(.ARM.Collect$$libinit$$00000021)
    .ARM.Collect$$libinit$$00000023          0x20000096   Section        0  libinit2.o(.ARM.Collect$$libinit$$00000023)
    .ARM.Collect$$libinit$$00000025          0x20000096   Section        0  libinit2.o(.ARM.Collect$$libinit$$00000025)
    .ARM.Collect$$libinit$$0000002C          0x20000096   Section        0  libinit2.o(.ARM.Collect$$libinit$$0000002C)
    .ARM.Collect$$libinit$$0000002E          0x20000096   Section        0  libinit2.o(.ARM.Collect$$libinit$$0000002E)
    .ARM.Collect$$libinit$$00000030          0x20000096   Section        0  libinit2.o(.ARM.Collect$$libinit$$00000030)
    .ARM.Collect$$libinit$$00000032          0x20000096   Section        0  libinit2.o(.ARM.Collect$$libinit$$00000032)
    .ARM.Collect$$libinit$$00000033          0x20000096   Section        2  libinit2.o(.ARM.Collect$$libinit$$00000033)
    .ARM.Collect$$libshutdown$$00000000      0x20000098   Section        2  libshutdown.o(.ARM.Collect$$libshutdown$$00000000)
    .ARM.Collect$$libshutdown$$00000002      0x2000009a   Section        0  libshutdown2.o(.ARM.Collect$$libshutdown$$00000002)
    .ARM.Collect$$libshutdown$$00000004      0x2000009a   Section        0  libshutdown2.o(.ARM.Collect$$libshutdown$$00000004)
    .ARM.Collect$$libshutdown$$00000006      0x2000009a   Section        0  libshutdown2.o(.ARM.Collect$$libshutdown$$00000006)
    .ARM.Collect$$libshutdown$$00000009      0x2000009a   Section        0  libshutdown2.o(.ARM.Collect$$libshutdown$$00000009)
    .ARM.Collect$$libshutdown$$0000000C      0x2000009a   Section        0  libshutdown2.o(.ARM.Collect$$libshutdown$$0000000C)
    .ARM.Collect$$libshutdown$$0000000E      0x2000009a   Section        0  libshutdown2.o(.ARM.Collect$$libshutdown$$0000000E)
    .ARM.Collect$$libshutdown$$00000011      0x2000009a   Section        0  libshutdown2.o(.ARM.Collect$$libshutdown$$00000011)
    .ARM.Collect$$libshutdown$$00000012      0x2000009a   Section        2  libshutdown2.o(.ARM.Collect$$libshutdown$$00000012)
    .ARM.Collect$$rtentry$$00000000          0x2000009c   Section        0  __rtentry.o(.ARM.Collect$$rtentry$$00000000)
    .ARM.Collect$$rtentry$$00000002          0x2000009c   Section        0  __rtentry2.o(.ARM.Collect$$rtentry$$00000002)
    .ARM.Collect$$rtentry$$00000004          0x2000009c   Section        6  __rtentry4.o(.ARM.Collect$$rtentry$$00000004)
    .ARM.Collect$$rtentry$$00000009          0x200000a2   Section        0  __rtentry2.o(.ARM.Collect$$rtentry$$00000009)
    .ARM.Collect$$rtentry$$0000000A          0x200000a2   Section        4  __rtentry2.o(.ARM.Collect$$rtentry$$0000000A)
    .ARM.Collect$$rtentry$$0000000C          0x200000a6   Section        0  __rtentry2.o(.ARM.Collect$$rtentry$$0000000C)
    .ARM.Collect$$rtentry$$0000000D          0x200000a6   Section        8  __rtentry2.o(.ARM.Collect$$rtentry$$0000000D)
    .ARM.Collect$$rtexit$$00000000           0x200000ae   Section        2  rtexit.o(.ARM.Collect$$rtexit$$00000000)
    .ARM.Collect$$rtexit$$00000002           0x200000b0   Section        0  rtexit2.o(.ARM.Collect$$rtexit$$00000002)
    .ARM.Collect$$rtexit$$00000003           0x200000b0   Section        4  rtexit2.o(.ARM.Collect$$rtexit$$00000003)
    .ARM.Collect$$rtexit$$00000004           0x200000b4   Section        6  rtexit2.o(.ARM.Collect$$rtexit$$00000004)
    .text                                    0x200000ba   Section        0  exit.o(.text)
    .text                                    0x200000cc   Section        8  libspace.o(.text)
    .text                                    0x200000d4   Section        2  use_no_semi.o(.text)
    .text                                    0x200000d6   Section        0  indicate_semi.o(.text)
    .text                                    0x200000d8   Section        0  sys_exit.o(.text)
    .ARM.__at_0x20000100                     0x20000100   Section        0  main.o(.ARM.__at_0x20000100)
    .text                                    0x200001ac   Section       78  rt_memclr_w.o(.text)
    .text                                    0x200001fa   Section       74  sys_stackheap_outer.o(.text)
    .text                                    0x20000244   Section       48  sys_stackheap.o(.text)
    .data                                    0x20000274   Section        8  main.o(.data)
    .bss                                     0x2000027c   Section     4668  main.o(.bss)
    SvsStack                                 0x2000027c   Data         512  main.o(.bss)
    __tagsym$$used                           0x2000027c   Number         0  main.o(.bss)
    .bss                                     0x200014b8   Section       96  libspace.o(.bss)

    Global Symbols

    Symbol Name                              Value     Ov Type        Size  Object(Section)

    BuildAttributes$$THM_ISAv4$P$D$K$B$S$PE$A:L22UL41UL21$X:L11$S22US41US21$IEEE1$IW$USESV6$~STKCKD$USESV7$~SHL$OSPACE$ROPI$EBA8$UX$STANDARDLIB$REQ8$PRES8$EABIv2 0x00000000   Number         0  anon$$obj.o ABSOLUTE
    __ARM_use_no_argv                        0x00000000   Number         0  main.o ABSOLUTE
    Image$$ZI$$Limit                          - Undefined Weak Reference
    __ARM_exceptions_init                     - Undefined Weak Reference
    __alloca_initialize                       - Undefined Weak Reference
    __arm_fini_                               - Undefined Weak Reference
    __arm_preinit_                            - Undefined Weak Reference
    __cpp_initialize__aeabi_                  - Undefined Weak Reference
    __cxa_finalize                            - Undefined Weak Reference
    __rt_locale                               - Undefined Weak Reference
    __sigvec_lookup                           - Undefined Weak Reference
    _atexit_init                              - Undefined Weak Reference
    _call_atexit_fns                          - Undefined Weak Reference
    _clock_init                               - Undefined Weak Reference
    _fp_trap_init                             - Undefined Weak Reference
    _fp_trap_shutdown                         - Undefined Weak Reference
    _get_lc_collate                           - Undefined Weak Reference
    _get_lc_ctype                             - Undefined Weak Reference
    _get_lc_monetary                          - Undefined Weak Reference
    _get_lc_numeric                           - Undefined Weak Reference
    _get_lc_time                              - Undefined Weak Reference
    _getenv_init                              - Undefined Weak Reference
    _handle_redirection                       - Undefined Weak Reference
    _init_alloc                               - Undefined Weak Reference
    _init_user_alloc                          - Undefined Weak Reference
    _initio                                   - Undefined Weak Reference
    _rand_init                                - Undefined Weak Reference
    _signal_finish                            - Undefined Weak Reference
    _signal_init                              - Undefined Weak Reference
    _terminate_alloc                          - Undefined Weak Reference
    _terminate_user_alloc                     - Undefined Weak Reference
    _terminateio                              - Undefined Weak Reference
    Reset_Handler                            0x20000001   Thumb Code    32  startup.o(.startup)
    _USAGEFAULT                              0x2000000d   Thumb Code     0  startup.o(.startup)
    NMI_Handler                              0x20000029   Thumb Code     2  startup.o(.startup)
    HardFault_Handler                        0x2000002b   Thumb Code     2  startup.o(.startup)
    MemManage_Handler                        0x2000002d   Thumb Code     2  startup.o(.startup)
    BusFault_Handler                         0x2000002f   Thumb Code     2  startup.o(.startup)
    UsageFault_Handler                       0x20000031   Thumb Code     2  startup.o(.startup)
    SVC_Handler                              0x20000033   Thumb Code     2  startup.o(.startup)
    DebugMon_Handler                         0x20000035   Thumb Code     2  startup.o(.startup)
    PendSV_Handler                           0x20000037   Thumb Code     2  startup.o(.startup)
    SysTick_Handler                          0x20000039   Thumb Code     2  startup.o(.startup)
    ADC1_2_IRQHandler                        0x2000003b   Thumb Code     0  startup.o(.startup)
    CAN1_RX1_IRQHandler                      0x2000003b   Thumb Code     0  startup.o(.startup)
    CAN1_SCE_IRQHandler                      0x2000003b   Thumb Code     0  startup.o(.startup)
    DMA1_Channel1_IRQHandler                 0x2000003b   Thumb Code     0  startup.o(.startup)
    DMA1_Channel2_IRQHandler                 0x2000003b   Thumb Code     0  startup.o(.startup)
    DMA1_Channel3_IRQHandler                 0x2000003b   Thumb Code     0  startup.o(.startup)
    DMA1_Channel4_IRQHandler                 0x2000003b   Thumb Code     0  startup.o(.startup)
    DMA1_Channel5_IRQHandler                 0x2000003b   Thumb Code     0  startup.o(.startup)
    DMA1_Channel6_IRQHandler                 0x2000003b   Thumb Code     0  startup.o(.startup)
    DMA1_Channel7_IRQHandler                 0x2000003b   Thumb Code     0  startup.o(.startup)
    EXTI0_IRQHandler                         0x2000003b   Thumb Code     0  startup.o(.startup)
    EXTI15_10_IRQHandler                     0x2000003b   Thumb Code     0  startup.o(.startup)
    EXTI1_IRQHandler                         0x2000003b   Thumb Code     0  startup.o(.startup)
    EXTI2_IRQHandler                         0x2000003b   Thumb Code     0  startup.o(.startup)
    EXTI3_IRQHandler                         0x2000003b   Thumb Code     0  startup.o(.startup)
    EXTI4_IRQHandler                         0x2000003b   Thumb Code     0  startup.o(.startup)
    EXTI9_5_IRQHandler                       0x2000003b   Thumb Code     0  startup.o(.startup)
    FLASH_IRQHandler                         0x2000003b   Thumb Code     0  startup.o(.startup)
    I2C1_ER_IRQHandler                       0x2000003b   Thumb Code     0  startup.o(.startup)
    I2C1_EV_IRQHandler                       0x2000003b   Thumb Code     0  startup.o(.startup)
    I2C2_ER_IRQHandler                       0x2000003b   Thumb Code     0  startup.o(.startup)
    I2C2_EV_IRQHandler                       0x2000003b   Thumb Code     0  startup.o(.startup)
    PVD_IRQHandler                           0x2000003b   Thumb Code     0  startup.o(.startup)
    RCC_IRQHandler                           0x2000003b   Thumb Code     0  startup.o(.startup)
    RTCAlarm_IRQHandler                      0x2000003b   Thumb Code     0  startup.o(.startup)
    RTC_IRQHandler                           0x2000003b   Thumb Code     0  startup.o(.startup)
    SPI1_IRQHandler                          0x2000003b   Thumb Code     0  startup.o(.startup)
    SPI2_IRQHandler                          0x2000003b   Thumb Code     0  startup.o(.startup)
    TAMPER_IRQHandler                        0x2000003b   Thumb Code     0  startup.o(.startup)
    TIM1_BRK_IRQHandler                      0x2000003b   Thumb Code     0  startup.o(.startup)
    TIM1_CC_IRQHandler                       0x2000003b   Thumb Code     0  startup.o(.startup)
    TIM1_TRG_COM_IRQHandler                  0x2000003b   Thumb Code     0  startup.o(.startup)
    TIM1_UP_IRQHandler                       0x2000003b   Thumb Code     0  startup.o(.startup)
    TIM2_IRQHandler                          0x2000003b   Thumb Code     0  startup.o(.startup)
    TIM3_IRQHandler                          0x2000003b   Thumb Code     0  startup.o(.startup)
    TIM4_IRQHandler                          0x2000003b   Thumb Code     0  startup.o(.startup)
    USART1_IRQHandler                        0x2000003b   Thumb Code     0  startup.o(.startup)
    USART2_IRQHandler                        0x2000003b   Thumb Code     0  startup.o(.startup)
    USART3_IRQHandler                        0x2000003b   Thumb Code     0  startup.o(.startup)
    USBWakeUp_IRQHandler                     0x2000003b   Thumb Code     0  startup.o(.startup)
    USB_HP_CAN1_TX_IRQHandler                0x2000003b   Thumb Code     0  startup.o(.startup)
    USB_LP_CAN1_RX0_IRQHandler               0x2000003b   Thumb Code     0  startup.o(.startup)
    WWDG_IRQHandler                          0x2000003b   Thumb Code     0  startup.o(.startup)
    __main                                   0x2000003d   Thumb Code     8  __main.o(!!!main)
    __scatterload                            0x20000045   Thumb Code     0  __scatter.o(!!!scatter)
    __scatterload_rt2                        0x20000045   Thumb Code    44  __scatter.o(!!!scatter)
    __scatterload_rt2_thumb_only             0x20000045   Thumb Code     0  __scatter.o(!!!scatter)
    __scatterload_null                       0x20000053   Thumb Code     0  __scatter.o(!!!scatter)
    __scatterload_zeroinit                   0x20000079   Thumb Code    28  __scatter_zi.o(!!handler_zi)
    __rt_lib_init                            0x20000095   Thumb Code     0  libinit.o(.ARM.Collect$$libinit$$00000000)
    __rt_lib_init_alloca_1                   0x20000097   Thumb Code     0  libinit2.o(.ARM.Collect$$libinit$$0000002E)
    __rt_lib_init_argv_1                     0x20000097   Thumb Code     0  libinit2.o(.ARM.Collect$$libinit$$0000002C)
    __rt_lib_init_atexit_1                   0x20000097   Thumb Code     0  libinit2.o(.ARM.Collect$$libinit$$0000001B)
    __rt_lib_init_clock_1                    0x20000097   Thumb Code     0  libinit2.o(.ARM.Collect$$libinit$$00000021)
    __rt_lib_init_cpp_1                      0x20000097   Thumb Code     0  libinit2.o(.ARM.Collect$$libinit$$00000032)
    __rt_lib_init_exceptions_1               0x20000097   Thumb Code     0  libinit2.o(.ARM.Collect$$libinit$$00000030)
    __rt_lib_init_fp_1                       0x20000097   Thumb Code     0  libinit2.o(.ARM.Collect$$libinit$$00000002)
    __rt_lib_init_fp_trap_1                  0x20000097   Thumb Code     0  libinit2.o(.ARM.Collect$$libinit$$0000001F)
    __rt_lib_init_getenv_1                   0x20000097   Thumb Code     0  libinit2.o(.ARM.Collect$$libinit$$00000023)
    __rt_lib_init_heap_1                     0x20000097   Thumb Code     0  libinit2.o(.ARM.Collect$$libinit$$0000000A)
    __rt_lib_init_lc_collate_1               0x20000097   Thumb Code     0  libinit2.o(.ARM.Collect$$libinit$$00000011)
    __rt_lib_init_lc_ctype_1                 0x20000097   Thumb Code     0  libinit2.o(.ARM.Collect$$libinit$$00000013)
    __rt_lib_init_lc_monetary_1              0x20000097   Thumb Code     0  libinit2.o(.ARM.Collect$$libinit$$00000015)
    __rt_lib_init_lc_numeric_1               0x20000097   Thumb Code     0  libinit2.o(.ARM.Collect$$libinit$$00000017)
    __rt_lib_init_lc_time_1                  0x20000097   Thumb Code     0  libinit2.o(.ARM.Collect$$libinit$$00000019)
    __rt_lib_init_preinit_1                  0x20000097   Thumb Code     0  libinit2.o(.ARM.Collect$$libinit$$00000004)
    __rt_lib_init_rand_1                     0x20000097   Thumb Code     0  libinit2.o(.ARM.Collect$$libinit$$0000000E)
    __rt_lib_init_return                     0x20000097   Thumb Code     0  libinit2.o(.ARM.Collect$$libinit$$00000033)
    __rt_lib_init_signal_1                   0x20000097   Thumb Code     0  libinit2.o(.ARM.Collect$$libinit$$0000001D)
    __rt_lib_init_stdio_1                    0x20000097   Thumb Code     0  libinit2.o(.ARM.Collect$$libinit$$00000025)
    __rt_lib_init_user_alloc_1               0x20000097   Thumb Code     0  libinit2.o(.ARM.Collect$$libinit$$0000000C)
    __rt_lib_shutdown                        0x20000099   Thumb Code     0  libshutdown.o(.ARM.Collect$$libshutdown$$00000000)
    __rt_lib_shutdown_cpp_1                  0x2000009b   Thumb Code     0  libshutdown2.o(.ARM.Collect$$libshutdown$$00000004)
    __rt_lib_shutdown_fini_1                 0x2000009b   Thumb Code     0  libshutdown2.o(.ARM.Collect$$libshutdown$$00000002)
    __rt_lib_shutdown_fp_trap_1              0x2000009b   Thumb Code     0  libshutdown2.o(.ARM.Collect$$libshutdown$$00000009)
    __rt_lib_shutdown_heap_1                 0x2000009b   Thumb Code     0  libshutdown2.o(.ARM.Collect$$libshutdown$$00000011)
    __rt_lib_shutdown_return                 0x2000009b   Thumb Code     0  libshutdown2.o(.ARM.Collect$$libshutdown$$00000012)
    __rt_lib_shutdown_signal_1               0x2000009b   Thumb Code     0  libshutdown2.o(.ARM.Collect$$libshutdown$$0000000C)
    __rt_lib_shutdown_stdio_1                0x2000009b   Thumb Code     0  libshutdown2.o(.ARM.Collect$$libshutdown$$00000006)
    __rt_lib_shutdown_user_alloc_1           0x2000009b   Thumb Code     0  libshutdown2.o(.ARM.Collect$$libshutdown$$0000000E)
    __rt_entry                               0x2000009d   Thumb Code     0  __rtentry.o(.ARM.Collect$$rtentry$$00000000)
    __rt_entry_presh_1                       0x2000009d   Thumb Code     0  __rtentry2.o(.ARM.Collect$$rtentry$$00000002)
    __rt_entry_sh                            0x2000009d   Thumb Code     0  __rtentry4.o(.ARM.Collect$$rtentry$$00000004)
    __rt_entry_li                            0x200000a3   Thumb Code     0  __rtentry2.o(.ARM.Collect$$rtentry$$0000000A)
    __rt_entry_postsh_1                      0x200000a3   Thumb Code     0  __rtentry2.o(.ARM.Collect$$rtentry$$00000009)
    __rt_entry_main                          0x200000a7   Thumb Code     0  __rtentry2.o(.ARM.Collect$$rtentry$$0000000D)
    __rt_entry_postli_1                      0x200000a7   Thumb Code     0  __rtentry2.o(.ARM.Collect$$rtentry$$0000000C)
    __rt_exit                                0x200000af   Thumb Code     0  rtexit.o(.ARM.Collect$$rtexit$$00000000)
    __rt_exit_ls                             0x200000b1   Thumb Code     0  rtexit2.o(.ARM.Collect$$rtexit$$00000003)
    __rt_exit_prels_1                        0x200000b1   Thumb Code     0  rtexit2.o(.ARM.Collect$$rtexit$$00000002)
    __rt_exit_exit                           0x200000b5   Thumb Code     0  rtexit2.o(.ARM.Collect$$rtexit$$00000004)
    exit                                     0x200000bb   Thumb Code    18  exit.o(.text)
    __user_libspace                          0x200000cd   Thumb Code     8  libspace.o(.text)
    __user_perproc_libspace                  0x200000cd   Thumb Code     0  libspace.o(.text)
    __user_perthread_libspace                0x200000cd   Thumb Code     0  libspace.o(.text)
    __I$use$semihosting                      0x200000d5   Thumb Code     0  use_no_semi.o(.text)
    __use_no_semihosting_swi                 0x200000d5   Thumb Code     2  use_no_semi.o(.text)
    __semihosting_library_function           0x200000d7   Thumb Code     0  indicate_semi.o(.text)
    _sys_exit                                0x200000d9   Thumb Code     8  sys_exit.o(.text)
    Region$$Table$$Base                      0x200000e4   Number         0  anon$$obj.o(Region$$Table)
    Region$$Table$$Limit                     0x200000f4   Number         0  anon$$obj.o(Region$$Table)
    _flash_program                           0x20000101   Thumb Code     8  main.o(.ARM.__at_0x20000100)
    _flash_erasepage                         0x20000109   Thumb Code     8  main.o(.ARM.__at_0x20000100)
    _flash_erasechip                         0x20000111   Thumb Code     8  main.o(.ARM.__at_0x20000100)
    _flash_readchip                          0x20000119   Thumb Code    10  main.o(.ARM.__at_0x20000100)
    main                                     0x20000123   Thumb Code   124  main.o(.ARM.__at_0x20000100)
    __aeabi_memclr4                          0x200001ad   Thumb Code     0  rt_memclr_w.o(.text)
    __aeabi_memclr8                          0x200001ad   Thumb Code     0  rt_memclr_w.o(.text)
    __rt_memclr_w                            0x200001ad   Thumb Code    78  rt_memclr_w.o(.text)
    _memset_w                                0x200001b1   Thumb Code     0  rt_memclr_w.o(.text)
    __user_setup_stackheap                   0x200001fb   Thumb Code    74  sys_stackheap_outer.o(.text)
    __user_initial_stackheap                 0x20000245   Thumb Code    48  sys_stackheap.o(.text)
    _RW_Limit                                0x20000270   Data           0  sys_stackheap.o(.text)
    errCnt                                   0x20000274   Data           4  main.o(.data)
    tMs                                      0x20000278   Data           4  main.o(.data)
    FlashParameter                           0x2000047c   Data        4156  main.o(.bss)
    __libspace_start                         0x200014b8   Data          96  libspace.o(.bss)
    __temporary_stack_top$libspace           0x20001518   Data           0  libspace.o(.bss)



==============================================================================

Memory Map of the image

  Image Entry point : 0x2000003d

  Load Region RAM (Base: 0x20000000, Size: 0x0000027c, Max: 0x00020000, ABSOLUTE)

    Execution Region CODE (Exec base: 0x20000000, Load base: 0x20000000, Size: 0x00000274, Max: 0x00010000, ABSOLUTE)

    Exec Addr    Load Addr    Size         Type   Attr      Idx    E Section Name        Object

    0x20000000   0x20000000   0x0000003c   Code   RO           26    .startup            startup.o
    0x2000003c   0x2000003c   0x00000008   Code   RO           35  * !!!main             c_w.l(__main.o)
    0x20000044   0x20000044   0x00000034   Code   RO          196    !!!scatter          c_w.l(__scatter.o)
    0x20000078   0x20000078   0x0000001c   Code   RO          198    !!handler_zi        c_w.l(__scatter_zi.o)
    0x20000094   0x20000094   0x00000002   Code   RO           62    .ARM.Collect$$libinit$$00000000  c_w.l(libinit.o)
    0x20000096   0x20000096   0x00000000   Code   RO           71    .ARM.Collect$$libinit$$00000002  c_w.l(libinit2.o)
    0x20000096   0x20000096   0x00000000   Code   RO           73    .ARM.Collect$$libinit$$00000004  c_w.l(libinit2.o)
    0x20000096   0x20000096   0x00000000   Code   RO           76    .ARM.Collect$$libinit$$0000000A  c_w.l(libinit2.o)
    0x20000096   0x20000096   0x00000000   Code   RO           78    .ARM.Collect$$libinit$$0000000C  c_w.l(libinit2.o)
    0x20000096   0x20000096   0x00000000   Code   RO           80    .ARM.Collect$$libinit$$0000000E  c_w.l(libinit2.o)
    0x20000096   0x20000096   0x00000000   Code   RO           83    .ARM.Collect$$libinit$$00000011  c_w.l(libinit2.o)
    0x20000096   0x20000096   0x00000000   Code   RO           85    .ARM.Collect$$libinit$$00000013  c_w.l(libinit2.o)
    0x20000096   0x20000096   0x00000000   Code   RO           87    .ARM.Collect$$libinit$$00000015  c_w.l(libinit2.o)
    0x20000096   0x20000096   0x00000000   Code   RO           89    .ARM.Collect$$libinit$$00000017  c_w.l(libinit2.o)
    0x20000096   0x20000096   0x00000000   Code   RO           91    .ARM.Collect$$libinit$$00000019  c_w.l(libinit2.o)
    0x20000096   0x20000096   0x00000000   Code   RO           93    .ARM.Collect$$libinit$$0000001B  c_w.l(libinit2.o)
    0x20000096   0x20000096   0x00000000   Code   RO           95    .ARM.Collect$$libinit$$0000001D  c_w.l(libinit2.o)
    0x20000096   0x20000096   0x00000000   Code   RO           97    .ARM.Collect$$libinit$$0000001F  c_w.l(libinit2.o)
    0x20000096   0x20000096   0x00000000   Code   RO           99    .ARM.Collect$$libinit$$00000021  c_w.l(libinit2.o)
    0x20000096   0x20000096   0x00000000   Code   RO          101    .ARM.Collect$$libinit$$00000023  c_w.l(libinit2.o)
    0x20000096   0x20000096   0x00000000   Code   RO          103    .ARM.Collect$$libinit$$00000025  c_w.l(libinit2.o)
    0x20000096   0x20000096   0x00000000   Code   RO          107    .ARM.Collect$$libinit$$0000002C  c_w.l(libinit2.o)
    0x20000096   0x20000096   0x00000000   Code   RO          109    .ARM.Collect$$libinit$$0000002E  c_w.l(libinit2.o)
    0x20000096   0x20000096   0x00000000   Code   RO          111    .ARM.Collect$$libinit$$00000030  c_w.l(libinit2.o)
    0x20000096   0x20000096   0x00000000   Code   RO          113    .ARM.Collect$$libinit$$00000032  c_w.l(libinit2.o)
    0x20000096   0x20000096   0x00000002   Code   RO          114    .ARM.Collect$$libinit$$00000033  c_w.l(libinit2.o)
    0x20000098   0x20000098   0x00000002   Code   RO          137    .ARM.Collect$$libshutdown$$00000000  c_w.l(libshutdown.o)
    0x2000009a   0x2000009a   0x00000000   Code   RO          147    .ARM.Collect$$libshutdown$$00000002  c_w.l(libshutdown2.o)
    0x2000009a   0x2000009a   0x00000000   Code   RO          149    .ARM.Collect$$libshutdown$$00000004  c_w.l(libshutdown2.o)
    0x2000009a   0x2000009a   0x00000000   Code   RO          151    .ARM.Collect$$libshutdown$$00000006  c_w.l(libshutdown2.o)
    0x2000009a   0x2000009a   0x00000000   Code   RO          154    .ARM.Collect$$libshutdown$$00000009  c_w.l(libshutdown2.o)
    0x2000009a   0x2000009a   0x00000000   Code   RO          157    .ARM.Collect$$libshutdown$$0000000C  c_w.l(libshutdown2.o)
    0x2000009a   0x2000009a   0x00000000   Code   RO          159    .ARM.Collect$$libshutdown$$0000000E  c_w.l(libshutdown2.o)
    0x2000009a   0x2000009a   0x00000000   Code   RO          162    .ARM.Collect$$libshutdown$$00000011  c_w.l(libshutdown2.o)
    0x2000009a   0x2000009a   0x00000002   Code   RO          163    .ARM.Collect$$libshutdown$$00000012  c_w.l(libshutdown2.o)
    0x2000009c   0x2000009c   0x00000000   Code   RO           37    .ARM.Collect$$rtentry$$00000000  c_w.l(__rtentry.o)
    0x2000009c   0x2000009c   0x00000000   Code   RO           39    .ARM.Collect$$rtentry$$00000002  c_w.l(__rtentry2.o)
    0x2000009c   0x2000009c   0x00000006   Code   RO           51    .ARM.Collect$$rtentry$$00000004  c_w.l(__rtentry4.o)
    0x200000a2   0x200000a2   0x00000000   Code   RO           41    .ARM.Collect$$rtentry$$00000009  c_w.l(__rtentry2.o)
    0x200000a2   0x200000a2   0x00000004   Code   RO           42    .ARM.Collect$$rtentry$$0000000A  c_w.l(__rtentry2.o)
    0x200000a6   0x200000a6   0x00000000   Code   RO           44    .ARM.Collect$$rtentry$$0000000C  c_w.l(__rtentry2.o)
    0x200000a6   0x200000a6   0x00000008   Code   RO           45    .ARM.Collect$$rtentry$$0000000D  c_w.l(__rtentry2.o)
    0x200000ae   0x200000ae   0x00000002   Code   RO           68    .ARM.Collect$$rtexit$$00000000  c_w.l(rtexit.o)
    0x200000b0   0x200000b0   0x00000000   Code   RO          119    .ARM.Collect$$rtexit$$00000002  c_w.l(rtexit2.o)
    0x200000b0   0x200000b0   0x00000004   Code   RO          120    .ARM.Collect$$rtexit$$00000003  c_w.l(rtexit2.o)
    0x200000b4   0x200000b4   0x00000006   Code   RO          121    .ARM.Collect$$rtexit$$00000004  c_w.l(rtexit2.o)
    0x200000ba   0x200000ba   0x00000012   Code   RO           55    .text               c_w.l(exit.o)
    0x200000cc   0x200000cc   0x00000008   Code   RO           63    .text               c_w.l(libspace.o)
    0x200000d4   0x200000d4   0x00000002   Code   RO          115    .text               c_w.l(use_no_semi.o)
    0x200000d6   0x200000d6   0x00000000   Code   RO          117    .text               c_w.l(indicate_semi.o)
    0x200000d6   0x200000d6   0x00000002   PAD
    0x200000d8   0x200000d8   0x0000000c   Code   RO          129    .text               c_w.l(sys_exit.o)
    0x200000e4   0x200000e4   0x00000010   Data   RO          194    Region$$Table       anon$$obj.o
    0x200000f4   0x200000f4   0x0000000c   PAD
    0x20000100   0x20000100   0x000000ac   Code   RO            1    .ARM.__at_0x20000100  main.o
    0x200001ac   0x200001ac   0x0000004e   Code   RO           33    .text               c_w.l(rt_memclr_w.o)
    0x200001fa   0x200001fa   0x0000004a   Code   RO           53    .text               c_w.l(sys_stackheap_outer.o)
    0x20000244   0x20000244   0x00000030   Code   RO           66    .text               c_w.l(sys_stackheap.o)


    Execution Region APP_RAM (Exec base: 0x20000274, Load base: 0x20000274, Size: 0x000012a4, Max: 0xffffffff, ABSOLUTE)

    Exec Addr    Load Addr    Size         Type   Attr      Idx    E Section Name        Object

    0x20000274   0x20000274   0x00000008   Data   RW            4    .data               main.o
    0x2000027c        -       0x0000123c   Zero   RW            2    .bss                main.o
    0x200014b8        -       0x00000060   Zero   RW           64    .bss                c_w.l(libspace.o)


==============================================================================

Image component sizes


      Code (inc. data)   RO Data    RW Data    ZI Data      Debug   Object Name

       172         14          0          8       4668       3728   main.o
        60         20          0          0          0        780   startup.o

    ----------------------------------------------------------------------
       232         34         28          8       4668       4508   Object Totals
         0          0         16          0          0          0   (incl. Generated)
         0          0         12          0          0          0   (incl. Padding)

    ----------------------------------------------------------------------

      Code (inc. data)   RO Data    RW Data    ZI Data      Debug   Library Member Name

         8          0          0          0          0         68   __main.o
         0          0          0          0          0          0   __rtentry.o
        12          0          0          0          0          0   __rtentry2.o
         6          0          0          0          0          0   __rtentry4.o
        52          8          0          0          0          0   __scatter.o
        28          0          0          0          0          0   __scatter_zi.o
        18          0          0          0          0         80   exit.o
         0          0          0          0          0          0   indicate_semi.o
         2          0          0          0          0          0   libinit.o
         2          0          0          0          0          0   libinit2.o
         2          0          0          0          0          0   libshutdown.o
         2          0          0          0          0          0   libshutdown2.o
         8          4          0          0         96         68   libspace.o
        78          0          0          0          0         80   rt_memclr_w.o
         2          0          0          0          0          0   rtexit.o
        10          0          0          0          0          0   rtexit2.o
        12          4          0          0          0         68   sys_exit.o
        48          8          0          0          0         80   sys_stackheap.o
        74          0          0          0          0         80   sys_stackheap_outer.o
         2          0          0          0          0         68   use_no_semi.o

    ----------------------------------------------------------------------
       368         24          0          0         96        592   Library Totals
         2          0          0          0          0          0   (incl. Padding)

    ----------------------------------------------------------------------

      Code (inc. data)   RO Data    RW Data    ZI Data      Debug   Library Name

       366         24          0          0         96        592   c_w.l

    ----------------------------------------------------------------------
       368         24          0          0         96        592   Library Totals

    ----------------------------------------------------------------------

==============================================================================


      Code (inc. data)   RO Data    RW Data    ZI Data      Debug   

       600         58         28          8       4764       4820   Grand Totals
       600         58         28          8       4764       4820   ELF Image Totals
       600         58         28          8          0          0   ROM Totals

==============================================================================

    Total RO  Size (Code + RO Data)                  628 (   0.61kB)
    Total RW  Size (RW Data + ZI Data)              4772 (   4.66kB)
    Total ROM Size (Code + RO Data + RW Data)        636 (   0.62kB)

==============================================================================

